:020000040000FA
:020000002F28A7
:08000800A000030EA1008B1AF9
:100010000B1D0D281F200B111A28831603138313A1
:100020000C1C1A288312031383130C1C1A282E206D
:100030000C101A28210E8300A00E200E09002E108D
:10004000AE14C201A303AC030800080008000800B6
:1000500008000800080008000612080008008501D2
:1000600086018316031383138D01843081002030B1
:1000700084008001840A041E392800308C00F0308E
:100080008500C0308600DB30870006309F00831279
:10009000031383133630920000309F00E0308B0052
:1000A0008514A901A91401221322A901C301012267
:1000B0006400AE1005142C08031D62284310430889
:1000C000A900012264008101871B622805108510A8
:1000D0006400AE185828871F68281E3001020318D4
:1000E00058286400AE185828871B71280108B000F2
:1000F00064008101871B78286400AE185828871F88
:100100007C281E300102031858286400AE185828B5
:10011000871B85280108B10064008101871B8C289A
:100120006400AE185828871F90281E30010203185B
:1001300058286400AE185828871B99280108B20077
:1001400064008101871BA0286400AE185828871F0F
:10015000A4281E300102031858286400AE1858283D
:10016000871BAD280108B30064008101871BB428F8
:100170006400AE185828871FB828203001020318E1
:1001800058286400AE185828871BC1280108B400FD
:1001900064008101871BC8286400AE185828871F97
:1001A000CC2820300102031858286400AE185828C3
:1001B000871BD5280108B500E1208921CC213F21EA
:1001C00058288101031003303C07A50030082502A0
:1001D000063C0318EE283008BC00B6003C08B60008
:1001E000031003303D07A50031082502063C031823
:1001F000FC283108BD00B7003D08B70003100330EC
:100200003E07A50032082502063C03180A293208D9
:10021000BE00B8003E08B800031003303F07A50039
:1002200033082502063C031818293308BF00B9001B
:100230003F08B900031003304007A5003408250229
:10024000063C031826293408C000BA004008BA004A
:10025000031003304107A50035082502063C0318AA
:1002600034293508C100BB004108BB001E30B6026E
:100270001E30B7021E30B8021E30B9020800A901B4
:100280002F303A0203185E2929303A02031C4C2908
:10029000291479290130AC0021303A02031C52297B
:1002A000A914792916303A02031C582929157929ED
:1002B0000A303A02031C5E29A91579292F303B0226
:1002C0000318862929303B02031C6829291679293D
:1002D00021303B02031C6E29A916792916303B02F6
:1002E000031C7429291779290A303B02031C792938
:1002F000A917AE1A7D29AE1608002E1A08002E1670
:1003000029084306A900C300012208002E12AE12DC
:1003100008008514051585158616ED3081002E140C
:1003200064002E18902981010F30C20001083602A6
:1003300003189C2985104210010837020318A229CE
:100340000511C210010838020318A82985114211AD
:10035000010839020318AE298612C2114208031D92
:10036000962985100511851186120800A7012D0810
:10037000A6000830A500A60C0318A70AA50BBB29E8
:10038000270803190800A7030800E130B000CC21BA
:1003900064002E19C82908000C3097003008B600F8
:1003A00083160313831364309200831203138313A1
:1003B00041303602031CEA293F303602A500031003
:1003C000A50DA50D250D143E9500061586112E15BB
:1003D000AE15FD29383036020318FB2936083A3CA1
:1003E000A5000310A50DA50D250D95000611861578
:1003F0002E15AE15FD299501AE1108002E1D970191
:1004000008002908A6000830A500261C092A861421
:100410000A2A861087168712A60CA50B052A061431
:100420000610861008000230A30064002308031D94
:10043000152A08002030A40064001322A40B1C2AF3
:020440000800B2
:02400E00763FFB
:00000001FF
